:100000000EC028C027C026C0DDC17CC123C022C0CD
:1000100021C020C05BC11EC01DC01CC01BC011245C
:100020001FBECFE5D1E0DEBFCDBF10E0A0E6B0E05F
:10003000E4E2F9E002C005900D92A837B107D9F7C4
:1000400010E0A8E7B0E001C01D92AC38B107E1F7BD
:100050004BD266C4D5CFC29890E087FF02C0C19A48
:1000600001C0C198C29A9F5FC298983011F0880F62
:10007000F4CF0895C09A88B3897F88BBC09808954B
:10008000109288001092890010928A0010928B00C2
:1000900008951F93182F87B3876087BB109289003C
:1000A00010928A0010928B0010938800812FD3DF6A
:1000B00010938900812FCFDF10938A00812FCBDF2F
:1000C00010938B00812FC7DFD5DF1F91089584E047
:1000D000809388008093890080938A0080938B00AE
:1000E000089580E4809388008093890080938A003B
:1000F00080938B0008958F929F92AF92BF92CF9280
:10010000DF92EF92FF920F931F93CF93DF934B01F8
:100110005C0120E030EC49E754ECACD2882314F4C5
:1001200080E40AC0C501B40120E03CE34CE156E4A0
:1001300088D3181654F484E0809388008093890053
:1001400080938A0080938B008CC0C501B40120E0AD
:1001500030E0A9018FD287FD02C010E005C0B7FAD8
:10016000B094B7F8B09411E0CC24C3940CC0C5018E
:10017000B4012DEC3CEC4CEC5DE367D3862E972E5E
:10018000A82EB92EC394C501B40120E030E040E2AE
:1001900051E457D387FFEBCFC501B4012FE632E11D
:1001A00043E05AE303D2062FF72EE82ED92E20E0A3
:1001B00030E040E251E445D3882374F0602F7F2D76
:1001C0008E2D9D2D2DEC3CEC4CEC5DE33ED3062FAB
:1001D000F72EE82ED92EC394C10E112321F081E011
:1001E0008093880011E0C12FDD27C7FDD095C85747
:1001F000DF4F602F7F2D8E2D9D2D40D2862F99278A
:1002000087FD90951C1569F4E12FFF27E7FDF09518
:10021000E857FF4F88599F4FDC018C9180618083A4
:1002200005C088599F4FFC01808188831F5F2196FC
:100230001430BCF4772767FD7095872F972F51D224
:100240009B01AC01602F7F2D8E2D9D2DAED120E026
:1002500030E040E251E4F9D2062FF72EE82ED92EF5
:10026000C8CFDF91CF911F910F91FF90EF90DF905A
:10027000CF90BF90AF909F908F900895F89488E1B1
:1002800081BD8FE081BD78940895F894A89514BE3F
:1002900088E181BD11BC7894089580EC8ABD8AEF15
:1002A00089BD84E083BF86E088BF89B7866189BF46
:1002B00081E080BF88B3886188BB10927E00109275
:1002C0007F00109280001092810008951F920F927B
:1002D0000FB60F9211248F9378948AB58F7B8ABDC5
:1002E00083B7806883BF8AB580648ABD88B386601F
:1002F00088BB87B3897F87BB8F910F900FBE0F900C
:100300001F9018951F920F920FB60F9211241F93F2
:100310002F933F934F935F936F937F938F939F930D
:10032000AF93BF93EF93FF93789486B386708093D7
:100330007D0087B3866087BB10917C001095109379
:100340007C0080918B00812786DE80918A00812746
:1003500082DE8091890081277EDE809188008F7EF9
:10036000812779DE20917D0080917B0090E0827072
:100370009070332727FD3095209530958223932365
:10038000009751F0F89410927E0010927F00109226
:10039000800010928100789480917D0080937B0092
:1003A000FF91EF91BF91AF919F918F917F916F914D
:1003B0005F914F913F912F911F910F900FBE0F9022
:1003C0001F9018951F920F920FB60F9211242F9322
:1003D0003F934F935F938F939F93AF93BF9386B356
:1003E000887190917800982780937800292F93FD49
:1003F00002C090E007C0882321F0883111F09FEF00
:1004000001C091E024FF08C0883009F449C0803160
:1004100009F446C09FEF02C09923D1F020917E00DD
:1004200030917F004091800050918100892F992761
:1004300087FD9095A92FB92F820F931FA41FB51F79
:1004400080937E0090937F00A0938000B093810002
:1004500078948091790090917A00019690937A0037
:100460008093790021E089339207E0F010927A00BE
:100470001092790080918300809184009091850092
:10048000A0918600B09187000196A11DB11D8093B7
:10049000840090938500A0938600B093870002C0EB
:1004A00091E0BCCFBF91AF919F918F915F914F91A0
:1004B0003F912F910F900FBE0F901F901895F894B9
:1004C00080917E0090917F00A0918000B09181008A
:1004D000789420917E0030917F004091800050916F
:1004E0008100B901CA010895BF92CF92DF92EF92C5
:1004F000FF920F931F9380E886BD16BCF89488E1A5
:1005000081BD8FE081BD789481E0C3DDC6DE789443
:1005100020E08FEF9FEFDC0100E2BB24B39403C027
:10052000D701C601212FA89505BF8895F894409161
:100530007E0050917F0060918000709181007894DE
:10054000C0907E00D0907F00E0908000F09081000D
:1005500010917D001470121711F0B0928200C8162D
:10056000D906EA06FB0621F4809182008823C1F2B5
:1005700010928200C701B601B4D020917D0022FF05
:1005800009C020916000309161004091620050915B
:10059000630008C0209164003091650040916600BE
:1005A0005091670052D1A7DDBBCF5058BB27AA2777
:1005B0000ED00DC1FED030F003D120F031F49F3FBA
:1005C00011F41EF4F3C00EF4E095E7FBE9C0E92F47
:1005D0000FD180F3BA17620773078407950718F0E5
:1005E00071F49EF527C10EF4E0950B2EBA2FA02DC5
:1005F0000B01B90190010C01CA01A0011124FF27D0
:10060000591B99F0593F50F4503E68F11A16F040CA
:10061000A22F232F342F4427585FF3CF46953795C9
:100620002795A795F0405395C9F77EF41F16BA0B8E
:10063000620B730B840BBAF09150A1F0FF0FBB1F3C
:10064000661F771F881FC2F70EC0BA0F621F731F85
:10065000841F48F4879577956795B795F7959E3FE2
:1006600008F0B3CF9395880F08F09927EE0F979570
:100670008795089571D008F481E0089504D06894B6
:10068000B111D9C00895BCD088F09F5790F0B92F10
:100690009927B751A0F0D1F0660F771F881F991FD7
:1006A0001AF0BA95C9F712C0B13081F0C3D0B1E0E9
:1006B0000895C0C0672F782F8827B85F39F0B93FF9
:1006C000CCF3869577956795B395D9F73EF49095D9
:1006D0008095709561957F4F8F4F9F4F0895E89457
:1006E00009C097FB3EF490958095709561957F4F7A
:1006F0008F4F9F4F9923A9F0F92F96E9BB27939528
:10070000F695879577956795B795F111F8CFFAF437
:10071000BB0F11F460FF1BC06F5F7F4F8F4F9F4F68
:1007200016C0882311F096E911C0772321F09EE8C6
:10073000872F762F05C0662371F096E8862F70E02C
:1007400060E02AF09A95660F771F881FDAF7880F06
:100750009695879597F90895990F0008550FAA0B5C
:10076000E0E8FEEF16161706E807F907C0F01216C4
:100770001306E407F50798F0621B730B840B950BC7
:1007800039F40A2661F0232B242B252B21F408951C
:100790000A2609F4A140A6958FEF811D811D0895B9
:1007A00097F99F6780E870E060E008959FEF80EC24
:1007B000089500240A9416161706180609060895C7
:1007C00000240A9412161306140605060895092E2D
:1007D0000394000C11F4882352F0BB0F40F4BF2B9C
:1007E00011F460FF04C06F5F7F4F8F4F9F4F0895DC
:1007F00057FD9058440F551F59F05F3F71F04795D2
:10080000880F97FB991F61F09F3F79F087950895B6
:10081000121613061406551FF2CF4695F1DF08C0D5
:10082000161617061806991FF1CF869571056105F2
:1008300008940895E894BB2766277727CB0197F99A
:1008400008958ADF08F48FEF08950AD0C0CFB1DF92
:1008500028F0B6DF18F0952309F0A2CFA7CFEBCF91
:10086000C7DFA8F39923D9F35523C9F3950F50E0B7
:10087000551FAA27EE27FF27BB270024089467955A
:1008800020F4E20FF31FB41F0A1E220F331F441F70
:10089000AA1F6695A9F7779530F4F30FB41F0A1EC7
:1008A000121E08F46395330F441FAA1F221F76956A
:1008B00099F7879520F4B40F0A1E121E631F440F88
:1008C000AA1F221F331F8695A9F7862F712D602D31
:1008D00011249F5750408AF0E1F088234AF0EE0F30
:1008E000FF1FBB1F661F771F881F91505040A9F73D
:1008F0009E3F510570F054CF9ECF5F3FECF3983E82
:10090000DCF3869577956795B795F795E7959F5FA3
:10091000C1F7FE2B880F911D9695879597F908953D
:04092000F894FFCF79
:100924000000803F0000803EEE886DCD8BC7E78CD1
:08093400EFCFAFE366E967278E
:00000001FF
